:020000040000FA
:1000000007309F008316F03085000F308600810096
:1000100083128501203086000514282005100C303D
:100020001D2028301D2001301D203030B400B500C7
:10003000B7003130B600B8013B28B2008600051485
:1000400028200510320E860005142820051008000F
:10005000B0012D20B00F29280800F030B100B10FF9
:100060002F280800B0013720B00F33280800B10155
:10007000B10F3828080083301D20B30185144520B6
:10008000FF39031954281D203F283308B30A82077B
:1000900055346C34743472346134203473346F34B6
:1000A0006E346934633400348510C5301D20B301CB
:1000B00085145F20FF39031969281D20592833084A
:1000C000B30A8207723461346E3467346534723433
:1000D0000034851095301D20B30185147420FF393C
:1000E00003197F281D206E283308B30A8207413484
:1000F0007534743468346F3472343A340034851093
:10010000D2301D20B30185148A20FF3903199A28A3
:100110001D2084283308B30A8207483465346E34BE
:1001200063347A34653420344734613462346F3454
:100130007234003406199A28F030B300851032204A
:1001400018301D20B30F9F280619A42801301D2048
:1001500084301D20B3018514B220FF390319BF2854
:100160001D20AC283308B30A820744346934733441
:10017000743461346E34633465343A34003440305E
:10018000B30004308506003E003E003E003E003EC7
:10019000003E003E003E003E003E003E003E003E6F
:1001A000003E003E003E003E003E003E003E003E5F
:1001B000003E003E003E003E003E003E003E003E4F
:1001C000003E003E003E003E003E003E003E003E3F
:1001D000003E003E003E003E003E003E003E003E2F
:1001E000B30BC128051E16290530B300B30BF62842
:1001F0003814B40A3408C63E031DF2283030B40067
:10020000B50A3508C63E031DF2283030B500B60ADF
:100210003608C63E031DF2283030B600B70A37084C
:10022000C63E031DF2283030B7004429381C62292D
:100230008510C2301D20851420301D2020301D2047
:100240003708303C0319272937081D202929203079
:100250001D2036081D2035081D202C301D20340897
:100260001D2020301D2063301D206D301D202030CA
:100270001D2020301D2085103030B400B500B7009F
:100280003130B6003810BF288510C2301D208514CB
:1002900020301D204F301D2076301D2065301D2060
:1002A00072301D2020301D2072301D2061301D2035
:1002B0006E301D2067301D2065301D2020301D2030
:1002C0008510BF288510C2301D2085144C301D209C
:1002D0006F301D2077301D2020301D2064301D2000
:1002E00069301D2073301D2074301D2061301D20A9
:1002F0006E301D2063301D2065301D208510BF2805
:02400E00623F0F
:00000001FF
